:020000001B28BB
:080008001B2863308C000C2062
:100010008D0B052800000800000000000000000013
:100020000000000000008C0B0C28000008000F08E6
:100030008D000520080083160030810000308B0001
:100040008316003085004330860081178312030138
:1000500085008600FA309000AA3091009630920018
:10006000FA30920005148510051106308D00052028
:1000700005148514051106308D0005200510851422
:10008000051105308D000520051085140515053076
:100090008D00052005108510051505308D00052003
:1000A00005148510051505308D000520900B3228AC
:1000B00005148510051103308D00052000308500E2
:1000C00005308D00052005108514051103308D00C5
:1000D00005200030850005308D00052005108510B5
:1000E000051503308D0005200030850005308D009A
:1000F0000520910B582805148510051103308D003B
:1001000005200030850003308D0005200510851482
:10011000051103308D0005200030850003308D006F
:10012000052005108510051503308D0005200030D1
:10013000850003308D000520920B7B280514851067
:10014000051103308D0005200030850002308D0040
:10015000052005108514051103308D0005200030A1
:10016000850002308D00052005108510051503302F
:100170008D0005200030850002308D000520900B99
:100180009E2805148510051102308D0005200030D1
:10019000850002308D000520051085140511023000
:1001A0008D0005200030850002308D0005200510EF
:1001B0008510051502308D000520003085000230C5
:0601C0008D000520C1289E
:00000001FF
